:1000000000308A00AE2800000000F73065000030A4
:10001000051901300038031D0F2811141116D228BC
:100020008E0A3C300E02031C21288E018F0A3C30C0
:100030000F02031C21288F01900A183010020318A8
:100040009001D82814088900831608148312080820
:1000500095000A301502031C3328203015020318BE
:100060003328063095021A301502031C39280C304B
:1000700095020130140797001708890083160814A9
:100080008312080896000A301602031C4D282030FF
:10009000160203184D28063096021A301602031C69
:1000A00053280C30960200341108403900380319E7
:1000B0007C28940114088900831608148312080808
:1000C0008C000C0A03197C28222015081002031D3D
:1000D000792816080F02031D7928023014079700AB
:1000E000170889008316081483120808FF3A03389A
:1000F0008600033094075A28D92817308400000856
:1001000003198A2888280000000000000000000071
:10011000800B83289628930A12081302031D9A283D
:10012000003066000610643097007D2800306600BD
:1001300006149301DA281108013900380319AD2893
:100140003E30940022201508900016088F008E0182
:1001500011179112111003309200DB2884018301E2
:1001600004308C008C1DBC28073081018130840054
:100170000008C0390F388000640081308400000816
:10018000C0390C0480000030660006109101013077
:10019000920093018101123090008F018E010B19A2
:1001A000D3280528CF280B110030660086171028A9
:1001B00054288B289B28003066008613CF286300C4
:02400E00F83F79
:00000001FF
